:020000040000FA
:10000000A0260020F9020000010300000303000005
:1000100005030000070300000903000000000000C2
:100020000000000000000000000000000B030000C2
:100030000D030000000000000F030000110300008A
:100040001303000013030000550800001303000011
:10005000130300001303000013030000A1030000BA
:100060000508000013030000130300001303000041
:100070001303000013030000130300001303000028
:100080001303000013030000130300001303000018
:100090001303000013030000130300001303000008
:1000A00013030000130300001303000013030000F8
:1000B0001303000013030000000000000000000014
:1000C00013030000130300001303000013030000D8
:1000D00013030000130300001303000000000000DE
:1000E0000000000000000000000000000000000010
:1000F0000000000000000000000000000000000000
:1001000000000000000000000000000000000000EF
:1001100000000000000000000000000000000000DF
:1001200000000000000000000000000000000000CF
:1001300000000000000000000000000000000000BF
:1001400000000000000000000000000000000000AF
:10015000000000000000000000000000000000009F
:10016000000000000000000000000000000000008F
:10017000000000000000000000000000000000007F
:10018000000000000000000000000000000000006F
:10019000000000000000000000000000000000005F
:1001A000000000000000000000000000000000004F
:1001B000000000000000000000000000000000003F
:1001C000000000000000000000000000000000002F
:1001D000000000000000000000000000000000001F
:1001E000000000000000000000000000000000000F
:1001F00000000000000000000000000000000000FF
:10020000DFF80CD000F0BAF800480047550D0000A8
:10021000A026002030B4044654E8000F0D4644E800
:100220000053002BF8D1156030BC704730B4044641
:1002300054E8000F40EA010544E80053002BF7D1D1
:10024000156030BC704730B4044654E8000F00EA33
:10025000010544E80053002BF7D1156030BC70470E
:1002600030B4044654E8000F80EA010544E8005326
:10027000002BF7D1156030BC704730B4044654E809
:10028000000F00EB010544E80053002BF7D1156087
:1002900030BC704730B4044654E8000FA0EB0105B1
:1002A00044E80053002BF7D1156030BC704770B4A0
:1002B00004464FF0000054E8006F0D68AE4207BFDF
:1002C00044E80023012044E800630E60002B1CBFBB
:1002D0000020F0E770BC704730B4044654E8000FCB
:1002E00088422CBF451A054644E80053002BF5D13F
:1002F000156030BC7047000006488047064800473C
:10030000FEE7FEE7FEE7FEE7FEE7FEE7FEE7FEE7C5
:10031000FEE7FEE7E9040000010200000048704724
:100320009C2F000040EA01039B0703D009E008C9A5
:10033000121F08C0042AFAD203E011F8013B00F8AA
:10034000013B521EF9D27047D2B201E000F8012BF6
:10035000491EFBD270470022F6E710B513460A4645
:1003600004461946FFF7F0FF204610BD421C10F866
:10037000011B0029FBD1801A70470000064C074D75
:1003800006E0E06840F0010394E807009847103465
:10039000AC42F6D3FFF738FF1034000030340000D1
:1003A0002DE9FE434FF48278404601F025FB4C4F87
:1003B00000254C4C012600B3404601F025FB94F883
:1003C0002E0010B194F82F10D1B18DF80050616853
:1003D00001912189ADF80810E26832B1218B618367
:1003E00062602181E56010B102E0257400E03E60AA
:1003F00021686846884784F82F5094F82E0060B32F
:100400004FF48077384601F0F7FA30B3384601F000
:10041000FBFA628B94F82D108A420AD9A2EB0100F4
:1004200080B260832289A2EB0000626802EB400088
:1004300005E007D1E06828B184F82F60658301F0FA
:10044000C9FA04E08A4202D184F82F6065834046ED
:1004500001F0DAFA2248001D06604FF4887738462A
:1004600001F0CAFA48B1384601F0CEFA25740220EC
:100470008DF800002168684688474FF48A7738462F
:1004800001F0BAFA28B1384601F0BEFA2574BDE889
:10049000FE834FF000484FF48C7967691DE000BF80
:1004A000B7FA87F028FA00F109EB80058F43284658
:1004B00001F0A2FA88B1284601F0A6FAA5F58C75DC
:1004C000E8088DF8040045F38000401C8DF80060BA
:1004D0008DF80500216868468847002FE0D1D6E7EF
:1004E00000700040E0000020F0B5B5480023021D78
:1004F0000178101D01254FF0805406290BD1167884
:10050000360708D10678C6F30316032E06D0042E4C
:1005100004D0052E02D0062907D00EE0B4F82463DB
:10052000A84FC6F304263E6002E01678360704D1D1
:100530000678C6F30316032E02D0062904D00FE076
:10054000A24FA14E7E670EE01678360708D10678D6
:10055000C6F30316032E06D0042E04D0052E02D0B7
:10056000062907D00EE0D4F84462994FC6F342360C
:100570003E6002E01678360704D10678C6F303160B
:10058000032E02D0062906D011E0924E376827F0DC
:10059000807737600EE01678360708D10678C6F304
:1005A0000316032E06D0042E04D0052E02D00629F1
:1005B0000AD011E04FF08046C6F80C31C6F8103171
:1005C000834E361F336002E01678360704D1067872
:1005D000C6F30316032E02D0062905D00CE07C4F8B
:1005E000032664373E600AE01678360704D10678A1
:1005F000C6F30316032E02D006290DD014E0764F61
:1006000005263E60744E78363560734E083633608A
:100610003F263F1D3E6002E01678360704D106787B
:10062000C6F30316052E02D0062957D062E06B4EA2
:1006300036686B4F3E60694E361D36683F1D3E6022
:10064000664E083636683F1D3E60644E0C3636688E
:100650003F1D3E60614E103636683F1D3E605F4E66
:10066000143636683F1D3E605C4E183636685C4F67
:1006700020373E60594E1C3636683F1D3E60574E4F
:10068000203636683F1D3E60544E243636683F1D86
:100690003E60524E283636683F1D3E604F4E2C3627
:1006A00036683F1D3E604D4E303636684C4F403701
:1006B0003E604A4E343636683F1D3E60474E3836FF
:1006C00036683F1D3E60454E3C3636683F1D3E60F5
:1006D000424E403636683F1D3E6002E016783607CF
:1006E00008D10678C6F30316032E06D0042E04D0D4
:1006F000052E02D0062907D019E0D4F85812394A3D
:1007000001F04F01116002E0117809070FD1007864
:10071000C0F30310032803D0042801D0052806D114
:1007200031480168C90702D06FF001010160D4F8B7
:100730003001062808D1D4F83401062804D12B480A
:10074000016841F48061016022487438016841F415
:1007500070010160BFF34F8FBFF36F8F4FF0102117
:10076000D1F80002002803DBD1F80402002822DAC5
:100770001F4A15601F480468002CFCD01524C1F8DE
:1007800000420568002DFCD0C1F804420168002930
:10079000FCD0136001680029FCD0BFF34F8F0D48D7
:1007A000F0380168144A01F4E06111430160BFF3BD
:1007B0004F8F00BFFDE7124910480860F0BD0000F0
:1007C000E00F00F0403501400DF0ADBA00C0074029
:1007D0003C050040FCED00E0105600400404001011
:1007E00020C50040E40E0040000400403C170040DB
:1007F00004E5014000E401400400FA050090D00344
:10080000A80000202DE9F047104E042700244FF4E3
:10081000A0784FF4803900BF08EB840509FA04F092
:10082000715961B1D6F80413014208D02946304607
:1008300001F032F90648D0E9002128469047641CAF
:10084000E4B2BC42E8D3BDE8F0870000008000407D
:10085000100100200148006800470000200000202F
:1008600002E008C8121F08C1002AFAD17047704779
:10087000002001E001C1121F002AFBD170470000D7
:1008800072B600F09FFF00BF00F0DAFD0028FBD138
:10089000104C0121208801EB00400FA100F0DCFE8C
:1008A00010480068C00700D000BE2088022101EB7C
:1008B00000400DA100F0D0FEBFF34F8F0948E4388F
:1008C00001680D4A01F4E06111430160BFF34F8FED
:1008D00000BFFDE7C8000020466174616C206572AE
:1008E000726F7200F0ED00E053797374656D2072E1
:1008F00065736574000000000400FA050EB5002160
:100900000091CDE901106A4644F20100FFF7B8FFFB
:100910000EBD00F003B800F009B8000072B602483E
:100920000168491C016070472800002003490868DD
:10093000401E086000D162B6704700002800002009
:100940002DE9F041064608680C46411C4FF0A047CF
:100950004FF0010506D005FA00F1C7F80815206828
:1009600000F082FC6068411C02D0002100F06AFCAB
:100970003168A069C1F82405607D227D316810438B
:10098000C1F86C05D4E900123068C0F81425C0F82D
:100990000C15207D012815D1A068411C02D0002132
:1009A00000F050FCE068411C05D08540C7F80855B0
:1009B000E06800F059FCD4E902123068C0F808255C
:1009C000C0F81015BDE8F0812DE9F0410646086831
:1009D0000C46411C4FF0A0474FF0010506D005FA28
:1009E00000F1C7F80815206800F048FC6068411C59
:1009F00002D0002100F02FFC3168A069C1F8240565
:100A0000607D217D32680843C2F86C05D4E900128C
:100A10003068C0F80C15C0F81425207D012815D1C8
:100A2000A068411C02D0002100F015FCE068411CC8
:100A300005D08540C7F80855E06800F01FFCD4E9F0
:100A400002123068C0F80825C0F81015BDE8F08122
:100A50002DE9F0470546861C90460F464FF00109E8
:100A60000020FFF756FF1B4C20683860D4E90001D6
:100A7000401AA16804F21C47081A0EE0012138460A
:100A800000F0FCF900F018F90146384600F0F6F9DC
:100A9000D4E90001401AA168081A401C8642EDD82A
:100AA000B8F1000F03D0052065F3891002E006209D
:100AB00065F39F50A2682168114004EB8101C86072
:100AC0002068304420600020FFF725FF4846BDE83D
:100AD000F08700007802002030B482680468531C5C
:100AE0008360A154D0E901128A4202D330BC00F0E5
:100AF0007ABA30BC70470000034803C8814201D174
:100B000001207047002070477802002010B50021B6
:100B1000024800F0BEF980F3100010BD94060020DA
:100B20002DE9FC5F0E008346DDE90C47C6F10000AD
:100B300098469246814600D40846012503E000BF4E
:100B400090FBFAF06D1C5045FADAA84500D94546ED
:100B500024B1002E01DB780700D5641EB80702D54A
:100B6000B8F1000F0AD0F80708D13CB1A54205D270
:100B700020215846641EFFF7AFFFF6E7002E02DA89
:100B80004E462D2102E0780703D52B215846FFF76A
:100B9000A3FF07F0030002280BD1B8F1000F08D122
:100BA0003CB1A54205D230215846641EFFF794FFA0
:100BB000F6E7CDE90047434652463146584601F034
:100BC000DFFFBDE8FC9F000070B50D4604460068DD
:100BD0004FF4887100F07CFF4FF49071206800F0B2
:100BE00077FF4FF49271206800F072FF4FF4A2710A
:100BF000206800F06DFF20681249C0F804132068D7
:100C00006907000B40B2090E002806DA00F00F0059
:100C100000F1E02080F8141D03E000F1E02080F8EE
:100C2000001420680121000B40B200F01F02914027
:100C30004009800000F1E020C0F88012C0F80011E7
:100C400070BD0000100302000246002012689307E6
:100C500002D0530702D47047500714D502F00300A6
:100C6000012802D002280CD105E0C2F383100B68E2
:100C7000801C184404E00223086803EB92521044DD
:100C8000086001207047086800EB9253C2F3891096
:100C9000401CEEE70121814003484068014201D039
:100CA000012070470020704718000020012181407A
:100CB000080300D0012070472DE9FF41002623489A
:100CC00000F0D9F82148001F074600F0D4F8204C66
:100CD00060680090A56800E000986946284004EB31
:100CE00080000C30FFF7B0FF0028F5D101AA009971
:100CF00001EA050304EB8303491CDB6842F820305A
:100D0000401C00910228F2D3019800F00300012852
:100D10000BD0022810D10198032101EB90500099CB
:100D2000BDF80A6001EB900005E00198BDF80A608B
:100D3000C0F3831008440090384600F099F808B1D9
:100D40000098606004B03046BDE8F0819006002055
:100D5000780200204FF40041002000F0EFFC08B1C1
:100D6000FFF7CCFD00F05EFB00F006FE08B1FFF7D8
:100D7000C5FD01F093FC01F0CBFC01F0BBFC084881
:100D80000321008801EB004006A100F065FC00BFD4
:100D900000F006FE00F054FB0028FBD1F8E700004D
:100DA000C800002053414144432048414C2073690E
:100DB0006D706C65206578616D706C652073746111
:100DC000727465642E0000002DE9F047C788044660
:100DD000181D16468946B0FBF7F1B0FBF7F207FB8A
:100DE00012009A193A44D21CB2FBF7F2DDF820A0A7
:100DF00001E02468491E0029FBD13D1A8846B5420E
:100E000016D818E0BAF1000F05D0211809EB080038
:100E10002A46091D04E0204409EB08012A46001D6A
:100E2000FFF780FA00202468761BA844B74201D956
:100E3000354600E03D46002EE4D1BDE8F0870000D5
:100E400030B5024659B100F0A5FC0021074C09E07D
:100E500004EB810315685B88AB4202D1116000206E
:100E600030BD491C8142F3D3052030BDAC000020C9
:100E7000002100F009B8012100F010B808B56A4659
:100E8000FFF7FBF9009808BD08B56A46FFF7DBF9E4
:100E900008BD08B56A46FFF7BDF908BD08B56A4642
:100EA000FFF7C4F9009808BD08B56A46FFF7F2F9E4
:100EB000009808BD70B5044600252846FFF729FDB7
:100EC00021686268086890420ED9401E0860017867
:100ED000A38AE26801FB0325227A2168101AC0B2B6
:100EE0000A79824200D208710020FFF714FD2846DB
:100EF00070BD70B505460C460020FFF70AFDE86896
:100F0000A98A201AB0FBF1F12A681068431C13600B
:100F10000170BDE870400020FFF7FDBC10B530B196
:100F2000017A42680368891AC9B21A6006E00E2085
:100F300010BD03681A68541C1C601170491EC9B2A8
:100F4000F7D2006800210171084610BD04480178FD
:100F500009B1852070470121017000207047000011
:100F600008000020F0B505460478154889B01646FB
:100F700040F82420124A0869121DA2F1080742F81D
:100F80002400487F385520226846FFF7CBF90494A7
:100F90002878385C48B10EB10A4A00E00022694660
:100FA000281D01F0B1F909B0F0BD0EB1064A00E00C
:100FB0000022694605F10C0001F078F8F3E7000023
:100FC000100000205D2A0000A92800000FB408B519
:100FD0000399002904D004AA00926A4600F00FF891
:100FE00001B05DF814FB10B582680446002A05D0F4
:100FF000D4E90403216898470020A06010BD2DE9C2
:10100000FC4791460C00804676D014F8011B39B19C
:1010100025290ED04046FFF75FFD20780028F4D147
:1010200098F80C00002867D04046BDE8FC47FFF761
:10103000DABF0020012221782B291BD02D2902D0D4
:10104000302908D102E040F0010001E040F0020048
:10105000641C002AEFD100252A290ED02178A1F1A5
:1010600030020A2A11D205EB850201EB4205641C0D
:10107000303DF1E740F00400EAE7D9F800100B1D1D
:10108000C9F800300968641C0D44217800232E291A
:101090000BD114F8011FA1F130020A2A05D203EB8B
:1010A000830201EB4203303BF3E76C290DD0682942
:1010B0000BD0692921D00BDC252918D0582931D033
:1010C00063290ED0642915D117E014F8011FECE74D
:1010D000702969D0732932D075291BD0782909D19C
:1010E00020E0D9F80000011DC9F800100178404641
:1010F000FFF7F2FC641C90E76CE0D9F800100A1DC1
:10110000C9F800200968CDE900500A224046FFF7DF
:1011100007FDEFE7D9F800100A1DC9F8002009689B
:101120000A2206E0D9F800100A1DC9F80020096853
:101130001022CDE90050404601F022FDDAE7D9F84F
:10114000001000270A1DC9F800200E68C00705D14D
:1011500012E04046761C7F1CFFF7BEFC3178002968
:10116000F7D104E0202140466D1EFFF7B5FCBD42DB
:10117000C0D9002DF6D1BDE74EB13046FFF7F6F8E5
:10118000074604E0202140466D1EFFF7A5FCBD4246
:1011900006D9002DF6D103E04046761CFFF79CFCF3
:1011A00031780029F8D1A5E7D9F80000011DC9F868
:1011B0000010056830214046FFF78EFC782140463C
:1011C000FFF78AFC08200021CDE900010346102228
:1011D0002946B0E7BDE8FC8770B541EA4201DDE988
:1011E00004564FF0A04441EA830141EA052104EB93
:1011F000800041EA0641C0F8001770BD70B541EAB1
:101200004201DDE904564FF0A04441EA830141EA7E
:10121000052104EB800041EA0641C0F8001770BDCB
:101220001CB5002100910B4601220191FFF7D4FF6C
:101230001CBD1CB5002100910B4601220191FFF756
:10124000DDFF1CBD1CB500220B4600921146019229
:10125000FFF7C2FF1CBD1CB500220B4600921146D1
:101260000192FFF7CBFF1CBD1CB5002100910B467E
:10127000012201911146FFF7AFFF1CBD1CB50021F3
:1012800000910B46012201911146FFF7B7FF1CBDEB
:1012900030B5124B01460020D3F81044224609E035
:1012A000157A854205D1401C0A28F7DB4FF0FF3044
:1012B00030BD5268002AF3D1421CF9D00872D3F82D
:1012C00010242AB152684A60D3F81024516030BD0E
:1012D0000022C3F810144A6030BD000078020020DC
:1012E000F0B595B01C4615460F4608461A9E00F00C
:1012F00021FB182109A8FFF72EF80E96CDE9095415
:101300000023082203A9384600F029FB059806901F
:10131000BDF81000ADF81C00BDF81200ADF81E00BD
:1013200000208DF821000398082600F00300012812
:1013300002D0022818D032E003983346850AC0F361
:10134000C2008DF8200003980FA9C0F38314A200F7
:10135000384600F004FB09A8009006AB22460FA90E
:10136000284600F043FA1AE00398840DC0F3C20047
:101370008DF82000082C01D2254600E008253346D0
:101380002A460FA9384600F0EAFA2E44641B09AB3E
:1013900006AA29460FA800F07BF9002CEAD13846AE
:1013A00000F0CEFA15B0F0BD7047012001F09ABAF6
:1013B000084810B50178084A515C19B1001D01F0C8
:1013C0002FF802E00C3000F03DFFBDE81040002097
:1013D00001F088BA380000200C00002008B5034A4C
:1013E00000924023024AFFF77BFF08BDA1270000BF
:1013F000780100200A4A012902EBC00007D0022927
:1014000007D0032907D0042907D000207047022005
:10141000704704207047007970474079704700009A
:101420003034000010B5FFF7C0FF04210348FFF778
:101430002FFF02490120487210BD00004C0000201F
:101440002DE9F0478CB0FFF757FB18B100200CB026
:10145000BDE8F087784C0020C4F81804BFF34F8F24
:1014600060680290A5684FF00008284004EB8000F7
:1014700008E021680298814201D86160E6E72840CF
:1014800004EB80000C3002A9FFF7DEFB0028F0D14E
:1014900003AB029901EA050204EB8202491CD268FF
:1014A00043F82020401C02910228F2D3039800F058
:1014B0000300022802D001284ED0A5E00398502254
:1014C000810D8946B2EB905F00D850210E4666F33D
:1014D0009F5003900831594800F0E3F9070078D095
:1014E00000F028FA4346082203A9384600F03DFAE6
:1014F000029908F1080A2940681A8000001D8642F6
:1015000023D94D4D0C3530B1C2B204EB8101301AF4
:1015100090460C3104E02946F2B200259046284658
:10152000C6B25346384600F020FA0AEB08032DB144
:10153000324629464FEA070000F017FA029909F1EE
:10154000030001EB900002903AE004EB8101534666
:10155000324638460C31EFE70398C0F38311062971
:1015600000D3062161F389100390C0F38310801C1F
:101570008100324800F095F9070045D000F0DAF913
:101580004346082203A9384600F0EFF908F108089D
:1015900000260FE00298434600EA0501401C04EBD8
:1015A00081010290042238460C3100F0DEF908F186
:1015B0000408761C0398C0F38310B042EAD847B100
:1015C000D4F81054D4F8180468B1384600F0B8F9CB
:1015D0002CE019E0687A012804D12A6828463946A7
:1015E000126890476D68002DF4D1384600F0A8F9D4
:1015F0000020FFF78EF9D4F8180408B9029860604B
:101600000020FFF788F911E0D4F8104404E02168C5
:101610002046896888476468002CF8D10848022170
:10162000008801EB004007A100F016F8FFF764FA0C
:1016300080F001000BE70000780200207034000009
:10164000C80000204261636B656E647320666C7530
:10165000736865640000000000231A4601F0C0B8FA
:1016600008B5012300926A4601F0BAF808BD1CB51E
:10167000CDE9002302236A4601F0B2F81CBD3EB555
:10168000069C8DE81C0003236A4601F0A9F83EBDC4
:101690002DE9F0470E4680461C46924608293ED862
:1016A00094F80C90002020731946104600F02EFF8D
:1016B0000025B54206D218F805201AA12046FFF7EA
:1016C00085FC03E019A12046FFF780FC6D1C082D66
:1016D000EFD317A12046FFF779FC0025B54210D2C1
:1016E00018F80570FEF71AFE0068C05D10F03E0F96
:1016F00001D03A4600E02E220EA12046FFF766FCFC
:1017000003E00DA12046FFF761FC6D1C082DE5D319
:1017100001222146504600F0DBFE84F80C90BDE823
:10172000F0870000202530327800000020202000C3
:101730007C0000002563000020000000104810B568
:10174000FF218160002101604160C0F81814C0F8D9
:10175000141480F820140B4800F0F0F800280DD184
:1017600009480A490A4B401AC108002003E000BF9B
:1017700023F82000401C8842FAD3002010BD00004E
:101780007802002070340000703400003034000013
:10179000AC00002002480349401AC008704700000E
:1017A000703400003034000013B56846FFF748FB82
:1017B00008B100201CBD0248009950F831001CBD42
:1017C0003034000070B508480125D0F8104480F886
:1017D000205405E06572216820464968884764689E
:1017E000002CF7D170BD0000780200202DE9FF47E2
:1017F00081460C9D00200C462F7B28739846164688
:101800002946184600F082FE072E42D2DFE806F095
:1018100004090F161F2A360049462846FFF7D6FB53
:1018200037E0494628462268FFF7D0FB31E0D4E98B
:10183000002349462846FFF7C9FB2AE0A06800902C
:10184000D4E9002349462846FFF7C0FB21E0D4E94C
:101850000201CDE90001D4E9002349462846FFF7FB
:10186000B5FB16E004F1080007C88DE80700D4E9CD
:10187000002349462846FFF7A9FB0AE004F10800C7
:101880000FC88DE80F00D4E9002349462846FFF72A
:101890009DFB00222946404600F01AFE2F73BDE84A
:1018A000FF872DE9F041858A80462D1F4819C01C0D
:1018B000B0FBF5F0C6B24046FFF7FCFA041E19D0A3
:1018C0000020207101206071E58000272546761EEA
:1018D000C4F800800BE04046FFF7ECFA60B1617994
:1018E000491C6171286005467F1CC0F80080B74222
:1018F000F1D32046BDE8F081204600F002F8002038
:10190000F8E72DE9F041457901466B1E002201E020
:101910000968521C9A42FBD30F680146002605E075
:1019200038460C68FFF7E5FA2146761CAE42F7D33D
:10193000BDE8F0810121001DFFF7A0BAFFF7EEBA64
:1019400010B504460121001DFFF7AEFA10F0FF0F9D
:1019500004D12046BDE81040FFF7D3BF10BD38B515
:1019600001240094FFF730FA38BD38B50024009404
:10197000FFF72AFA38BD0000064910B5002048706C
:10198000091D0860BFF35F8F0349044800F046F863
:10199000002010BD2C000020B42D00006C010020A0
:1019A00010B50020FEF7B5FFF1EE100A20F09F0001
:1019B000E1EE100ABFF35F8F05494020C1F88002B5
:1019C0000020FEF7A8FF20BF40BF20BF10BD0000D1
:1019D00004E000E0024A1060101D01607047000042
:1019E0002C760040030103481844C0F81425C0F8C1
:1019F000101570470070004002494058002800D080
:101A00000120704700700040034908B508440022D7
:101A100002600068009008BD007000400160096825
:101A20004160AFF3008010B5D0E9002153689942BE
:101A300001D1002104E0D1E90034A34202D01946CB
:101A4000816010BD08314160F0E700000C4A10B51C
:101A500002F58C730EE0991AC91001EBD17149108F
:101A600002EBC1010C68844201D90B4602E005D2A9
:101A700001F108029A42EED3002010BD486810BD63
:101A8000D42D000000B5FFF7E1FF002800D1014888
:101A900000BD0000C02D000008B500224250405893
:101AA000009008BD4058002800D00120704708B5BC
:101AB000002242504058009008BDD0F8040308406E
:101AC00000D0012070474058002800D00120704706
:101AD00008B5002242504058009008BD0121B1EBEA
:101AE000507F01D101207047002070472DE9F05F41
:101AF0000427204EDFF88090834600244FF0030A2D
:101B00004FF001080020FEF704FF08FA04F5354203
:101B100003D02046FFF7BEF8B8B10020FEF7FBFE69
:101B2000FFB104F10104AE43E4B2EBD13846FFF754
:101B3000A9FFB9F8001003460AEB01400F4A10A1B3
:101B4000FFF795FD3846BDE8F09F154908FA04F007
:101B500000274A68104348608BF800403846FEF77B
:101B6000DAFEB9F8001022460AEB01400DA1FFF79A
:101B700077FDDBE7FFFF0F00C8000020512C0000BD
:101B800046756E6374696F6E3A2025732C206572FA
:101B9000726F7220636F64653A2025732E00000017
:101BA00018000020416C6C6F636174656420636889
:101BB000616E6E656C3A2025642E00002DE9F843B5
:101BC00014460D0081462CD0002C2AD00026FFF7A9
:101BD0006DF8174F4FF00308002824D04846FFF750
:101BE00059F8002821D0134800EBC900C0F810555F
:101BF000C0F81445009439882B4608EB01404A464A
:101C00000DA1FFF73CFD3046FFF73CFF3988034646
:101C100008EB0140184A19A1FFF729FD3046BDE83D
:101C2000F8830E20FBE70726EDE70826EBE7000028
:101C3000C800002000F0014041737369676E65645D
:101C4000206368616E6E656C3A2025642C20657691
:101C5000656E7420656E6420706F696E743A20251D
:101C6000782C207461736B20656E6420706F696ED0
:101C7000743A2025782E00007E2C000046756E6395
:101C800074696F6E3A2025732C206572726F722012
:101C9000636F64653A2025732E00000070B504461A
:101CA00001260025A640FFF701F818B12046FEF7EF
:101CB000F1FF80B1094806602846FFF7E3FE0346BE
:101CC00007480321074A008801EB004006A1FFF7FF
:101CD000CEFC284670BD0825EEE7000004F5014063
:101CE000C8000020B32C000046756E6374696F6EE7
:101CF0003A2025732C206572726F7220636F6465C1
:101D00003A2025732E00000070B50D4600F04AFC05
:101D100004000FD00020FEF7FCFD207920B1002048
:101D2000FEF7F9FD112070BD012025602071002013
:101D3000FEF7F1FD002070BD10B500F033FC002867
:101D400002D000210160017110BD00002DE9F041B9
:101D5000254C064612200D46C4F808032348017C92
:101D6000022918D0027C01464FF4807891F82E1099
:101D7000012A12D00222C4F8042301270774466006
:101D800005810022C26021B3458390F82D103046B2
:101D9000FFF720FE25E0122002E0C2682AB10220EF
:101DA000C4F804031120BDE8F081C660058361B961
:101DB00047463846FFF720FE0028FAD03846FFF79E
:101DC00023FE29463046FFF705FE0220C4F804032F
:101DD00007E029463046FFF7FDFD4046FFF714FEB9
:101DE00027600020DFE7000000700040E0000020D6
:101DF00070B505462A480C46017C09B1112070BD1A
:101E00002179284E09B1012901D10021316000EB6F
:101E100045010A7F1AB910F82D2F521C0270E07983
:101E20000877207A487721786278302301F003011F
:101E300003EA02121143A2784FF4E06303EA02229C
:101E40001143E2784FF4805303EA023211432279BE
:101E50004FF4E02303EA0242114362794FF4801306
:101E600003EA02521143A2791B0103EA02620E4BFC
:101E70002846114303EB0012C2F81815227AE179C3
:101E8000FFF7B0FD227AE1792846FFF7ABFD207914
:101E900008B1012801D101203060002070BD000090
:101EA000E000002000750040007000402DE9F04186
:101EB0001E4C054694F82C0010B10820BDE8F081B6
:101EC00044F8101B1A4928780860091D68780860D2
:101ED000E878A0770127277700202070607760607E
:101EE000144EE0776FF00040C6F808034FF482709C
:101EF000FFF78AFDB015FFF787FDA8780E4940016E
:101F000081F800048020C91FC1F88002C1F80001D7
:101F10000220C6F80403A07F10B10120C6F8040314
:101F20000348F03807600020C8E70000E000002008
:101F3000F07500400070004007E000E0044890F8B1
:101F40002E0008B1002000E0042002490844704738
:101F5000E0000020007000402DE9F04106460D46EB
:101F60004FF4803400681746AC404BB14FF4A07179
:101F700001EB8501FFF790FD3068C0F8044301E0F4
:101F8000C0F80843306800EB8500C0F84075BDE834
:101F9000F0810000016801220A600079034A00EB29
:101FA000400002EB80000221017270471001002006
:101FB000F0B40468049E40F20115D4F800728D401C
:101FC000AF43C4F800720468D4F800521D43C4F84B
:101FD00000523346F0BCFFF7BFBF00002DE9F041CF
:101FE00004460E4600792C4900EB400001EB8007C7
:101FF000387A10B10820BDE8F0813A607068002599
:102000004FF4A078786006E008EB85012068FFF7C0
:1020100043FD6D1CEDB26079A842F5D82068F178D7
:10202000000B40B200284FEA411106DA00F00F0021
:1020300000F1E02080F8141D03E000F1E02080F8BA
:10204000001420680122000B40B200F01F0302FAC6
:1020500003F14009800000F1E020C0F88012C0F8D0
:10206000001120687178D0F8043561F30103C0F8DD
:1020700004352068B178D0F8083561F30103C0F861
:10208000083520683178D0F8103561F30303C0F8C3
:1020900010353A720020AEE71001002001490248D5
:1020A00000F048BC1C010020002000402DE9F04158
:1020B0000546007916460F4600EB40012D4A01EB1C
:1020C000C00102EB810494F82A1011B10820BDE888
:1020D000F081294951F820102868FFF715FE08B152
:1020E0001120F4E739462846FEF72AFC6660386975
:1020F000206030004FF001062FD03F7F4FF48E71EB
:102100002868FFF7D4FC4FF4A2712868FFF7CFFCD2
:1021100028681A49C0F8041328684FEA4711000BD1
:1021200040B2002806DA00F00F0000F1E02080F84D
:10213000141D03E000F1E02080F800142868000B73
:1021400040B200F01F0206FA02F14009800000F1DF
:10215000E020C0F88012C0F8001128680421C0F8FF
:1021600000150020A061E06184F8290044F8140FF4
:10217000A675ACE71C010020842D00008000020041
:102180002DE9F047054600790B4600EB400101EBD5
:10219000C000234901EB8004284600F043F810B149
:1021A0001120BDE8F0874FF00008C4F82080A3603C
:1021B000626184F828804FF48E764746314628685D
:1021C000FFF775FC28684FF00109C0F80890214618
:1021D000286800F04CFB606800BBD5F800A00EE05A
:1021E00094F8280008B10F2716E031465046FFF753
:1021F00059FC0028F4D02146504600F038FB216AF3
:1022000060698142F1D331462868FFF74BFC002812
:10221000F9D02868C0F80C90C4F814803846C0E79C
:102220001C010020007900EB400101EBC0000449D3
:1022300001EB80004069002800D0012070470000B9
:102240001C0100202DE9F047044600794FF00009F9
:1022500000EB400101EBC000254901EB800720683D
:10226000C0F80095786880B120682249C0F808134A
:1022700020680121000B40B200F01F02914040098C
:10228000800000F1E020C0F880112068D0F80C2513
:10229000D0F81485D0F80865D0F810554FF0FF310C
:1022A000C0F81415C0F80C152068C0F80815C0F85F
:1022B0001015501C02D01046FEF7B2FFB8F1FF3FD8
:1022C00002D04046FEF7ACFF681C02D02846FEF75D
:1022D000A7FF701C02D03046FEF7A2FF2068FFF770
:1022E0002BFD87F82A90C7F80490BDE8F08700001E
:1022F0001C010020840202000149024800F0C6BB14
:1023000048010020002000402DE9F0410546164616
:1023100000790F46154A00EBC00102EB810494F8E6
:10232000201011B10820BDE8F081114951F82010AA
:102330002868FFF7E9FC08B11120F4E73946284680
:10234000FEF742FB6660386920601EB1397F28467F
:10235000FEF73AFC28680821C0F800150020A061AB
:10236000E0610121606184F82010DCE74801002071
:10237000882D00002DE9F04704460E4600792049DB
:1023800000EBC00001EB800517463046FFF7A6FBC7
:1023900030B1204600F036F820B11120BDE8F087BA
:1023A0001020FBE76F61AE604FF490760027314656
:1023B0002068FFF78DFB4FF4AC7841462068FFF7AB
:1023C00087FB2068AA686969C0F84425C0F84815E9
:1023D000206801218160686878B9B1464946206863
:1023E000FFF771FB064641462068FFF76CFB06438A
:1023F000F4D000B10F27002068613846CEE7000016
:10240000480100200079054900EBC00001EB800085
:102410004069002800D001207047000048010020DA
:102420002DE9F04704460079274900EBC00001EB95
:10243000800720684FF00009C0F80095786880B1E7
:1024400020682249C0F8081320680121000B40B21F
:1024500000F01F0291404009800000F1E020C0F828
:1024600080112068D0F80C25D0F81485D0F80865C4
:10247000D0F810554FF0FF31C0F80C15C0F8141506
:102480002068C0F80815C0F81015501C02D010467E
:10249000FEF7CFFEB8F1FF3F02D04046FEF7C9FE7F
:1024A000681C02D02846FEF7C4FE701C02D03046DD
:1024B000FEF7BFFE2068FFF73FFC87F82090C7F8C3
:1024C0000490BDE8F08700004801002010030200DE
:1024D00010B50C46017A052908D0407A38B1084871
:1024E00008A102682046FEF771FD00E01AB106A1BE
:1024F0002046FEF76BFD2046BDE81040FEF773BD99
:1025000084000020257300000D0A000038B5C38840
:102510000D46044633B114A0009015A216A128461A
:10252000FEF754FD217A05291CD0607A48B1A088B5
:10253000FEF760FF164951F8202016A12846FEF745
:1025400045FDA0880021FFF72FF903461049207AA6
:10255000143951F8202001B02846BDE830400EA1C2
:10256000FEF734BD38BD00001B5B306D000000007D
:102570001B5B313B33316D0025734C6F67732064F7
:10258000726F70706564202825642925730D0A0018
:1025900084000020257300003C25733E2025733AFB
:1025A000200000000349884201D103487047002001
:1025B00070470000002000402000002070B5054654
:1025C00088690C4600284FF4847128460AD0FFF72A
:1025D0006EFAD5F81805626AE1688854606A401C92
:1025E000606270BDFFF763FAD5F8180570BD1FB5BE
:1025F00001238DF80030CDE90121D0E900126846B1
:1026000090471FBD1FB501238DF800308DF80810CD
:102610000192D0E90012684690471FBD2DE9F041B4
:1026200005460078002824D105216868FFF78EFB55
:1026300008B1FEF763F9104FDFF8408003263888B1
:102640000FA106EB0040D8F80420FFF709F800249A
:10265000686811A130F91420388806EB0040FEF7B5
:10266000FFFF641C052CF3DBD8F80410491CC8F8E4
:102670000410BDE8F0810000C80000200000002028
:10268000414443206576656E74206E756D62657297
:102690003A20256400000000256400000EB5124AAF
:1026A00007CA8DE80700104810491438FFF7FEFBF1
:1026B00008B1FEF723F969460020FFF799FB08B13E
:1026C000FEF71CF905210A48FFF740FB08B1FEF7A9
:1026D00015F9074805210A30FFF738FB002801D01B
:1026E000FEF70CF90EBD0000482C00001D2600006E
:1026F000CC000020054810B50078FFF7CFFA00287D
:1027000003D0BDE81040FEF7F9B810BD000000206E
:102710003EB5FEF71BFC08B1FEF7F0F81C491D4A58
:10272000D1E90301CDE9010103208DF80600184825
:1027300001A9001DFFF752FC08B1FEF7DFF8144CA9
:10274000241D2068D0F81005134A0123C240002040
:10275000014600902046FFF72BFC2046FFF71AFCAD
:10276000246804F5A074FFF7E9FB05460B48FFF762
:10277000BDF908B1FEF7C2F808482A46214600789C
:10278000FFF71CFA002801D0FEF7B8F83EBD0000A4
:10279000342C00006D28000000A86100000000201B
:1027A00070B50D4C0020D2B22070201D0B4D037867
:1027B000EB5C1BB1001DFFF7DDFD02E00C30FFF705
:1027C000DFFC08B1FEF79AF86078002802D0217883
:1027D0000029FAD070BD0000340000200C00002059
:1027E0002DE9F84F204D924689460646984601222B
:1027F00069461846AF68FEF72BF958B300980021D8
:102800000446801C09E000BF00EA07035AF82120B3
:1028100005EB8303401C491CDA604145F4D34FEAC1
:10282000164AFEF773F94AEA0041601C384005EB8E
:1028300080003C4005EB8402C160D06866F3C500AF
:1028400068F3891069F39F2020F00300401C20F0FA
:102850000400D06095F8200402E000BFFEF7F0FD10
:102860000028FBD1BDE8F88F78020020704770B5D2
:102870000C4605464FF48E71FFF719F9216AA068DE
:10288000415C206A401C2062C5F81C1570BD1FB554
:1028900000228DF800200291816801914261D0E907
:1028A0000012684690471FBD1FB50A4601788DF893
:1028B000001041680191017A8DF80810C0680390FA
:1028C000044850F82210001F50F822206846904714
:1028D0001FBD00001400002001490120087070474E
:1028E0003400002010B588B0044620220E49684606
:1028F000FDF718FD06200090C01F01900290039084
:102900004FF0EB7006900CB1084A00E000226946D7
:102910000748FEF727FB08B1FDF7F0FF0448001F4A
:10292000447008B010BD0000F82E0000D928000047
:10293000380000202DE9FF470C4605464FF4007192
:10294000FFF7BBF801274FF40178002618B34FF4C6
:10295000927949462846FFF7A5F8E0B1494628464E
:10296000FFF7A5F8C5F8088394F8290000B96F604F
:1029700002208DF80000D5F88004C5F8800403908B
:10298000A0690290E0680190A661E661D4E90012B6
:102990006846904728E004212846FFF78EF818B3D0
:1029A0004FF484712846FFF77DF8E8B121462846A8
:1029B000FFF704FE616AA069884215D1E06938B169
:1029C000E268616AA0612069E6616662E06008E031
:1029D00094F8290000B96F60C5F80883A661E26821
:1029E000616A2046FFF703FE4FF48E784146284681
:1029F000FFF758F878B1206A6169884202D294F8EA
:102A0000280020B341462846FFF751F8616911B10B
:102A10002046FFF73CFF4FF4A27841462846FFF7D7
:102A200041F8002818D041462846FFF740F894F8AE
:102A3000290000B12F60A06900280DD0A661E268CE
:102A4000616A04B02046BDE8F047FFF7D0BD2146DB
:102A50002846FFF70CFFDEE7BDE8FF871FB50A46F3
:102A600001788DF8001041680191017A8DF8081005
:102A7000C0680390044850F82210001F50F822202C
:102A8000684690471FBD0000140000202DE9FF415B
:102A90000C464FF4927705463946FFF714F80026A6
:102AA000C0B139462846FFF713F802208DF8000020
:102AB000D5F88004C5F880040390D5F83C058DF85E
:102AC0000800E0680190A661E661D4E9001268465A
:102AD000904723E04FF4887739462846FEF7F3FF06
:102AE000E0B139462846FEF7F3FFD5F83C15A0695A
:102AF000884213D1E06960B1E268D5F8000220F0A5
:102B00002000C5F80002E069A0612069E661E0608C
:102B100001E0A661E2682046FFF774FD4FF4A2775A
:102B200039462846FEF7CFFF60B139462846FEF702
:102B3000CFFFA06930B1A661D5F83C152046E26808
:102B4000FFF760FD4FF4907739462846FEF7BBFF4C
:102B5000002813D039462846FEF7BAFF60690028DE
:102B60000CD0D5F84C058DF800608DF80800A068F1
:102B700001906661D4E9001268469047BDE8FF8184
:102B80002DE9F05F8346DDE90A4A994690460D46F5
:102B90000846012703E000BFB0FBF8F07F1C40456A
:102BA000FAD2B94500D94F465FEACA7012D18CB14A
:102BB0005FEA8A7002D5B9F1000F01D0202607E044
:102BC000302605E031465846641EFDF785FF0CB1FE
:102BD000A742F7D35FF00106B9F1010F02D9A9F1BD
:102BE000010903E0B5FBF6F0404502D306FB08F609
:102BF000F2E7DFF83C9000BFB5FBF6F000FB16559E
:102C000019F800105846FDF767FFB6FBF8F6002EDE
:102C1000F2D15FEACA7009D0002C07D0A74205D2D2
:102C200020215846641EFDF757FFF5E7BDE8F09FE9
:102C30008C2D00000100070000800040000400000F
:102C4000000000070000000000000000020000017A
:102C5000006E7266785F7070695F6368616E6E6542
:102C60006C5F616C6C6F63006E7266785F70706928
:102C70005F6368616E6E656C5F66726565006E723B
:102C800066785F7070695F6368616E6E656C5F61C6
:102C9000737369676E006E7266785F7070695F63E8
:102CA00068616E6E656C5F666F726B5F617373698E
:102CB000676E006E7266785F7070695F6368616EE0
:102CC0006E656C5F656E61626C65006E7266785FE2
:102CD0007070695F6368616E6E656C5F6469736173
:102CE000626C65006E7266785F7070695F67726FA4
:102CF00075705F616C6C6F63006E7266785F707088
:102D0000695F67726F75705F66726565006E726687
:102D1000785F7070695F67726F75705F656E616212
:102D20006C65006E7266785F7070695F67726F7550
:102D3000705F64697361626C65006E7266785F7063
:102D400070695F6368616E6E656C735F72656D6FED
:102D500076655F66726F6D5F67726F7570006E7219
:102D600066785F7070695F6368616E6E656C735FD3
:102D7000696E636C7564655F696E5F67726F7570AD
:102D8000000000009D200000F922000030313233A5
:102D90003435363738394142434445460000000057
:102DA0000000000000000000000000000000000023
:102DB000000000009C2D0000B42D00000400000065
:102DC000556E6B6E6F776E206572726F7220636FD7
:102DD00064650000000000000433000001000000F2
:102DE000C431000002000000B82F00000300000002
:102DF00038320000040000008C32000005000000A2
:102E00006C310000060000000831000007000000DF
:102E1000743200000800000080310000090000004A
:102E2000E43100000A000000EC3200000B0000005A
:102E3000A02F00000C000000983100000D000000E1
:102E40003C3300000E000000643200000F00000060
:102E5000A032000010000000D43200001100000079
:102E6000503300008000000020310000810000008D
:102E70005C300000820000001C3000008300000075
:102E8000FC2F0000840000003830000085000000A6
:102E900044310000860000004C3200009000000029
:102EA000E830000091000000DC2F000092000000DC
:102EB000AC31000000820000B4320000018200004A
:102EC00000320000028200001C320000008400007A
:102ED00078300000018400001033000002840000FC
:102EE000C0300000038400009C300000DD130000AF
:102EF000B1130000A9130000FFFFFFFFFFFFFFFF5A
:102F0000FFFFFFFFFFFFFFFF0000000000000000C9
:102F10000000D60107010000004040404040404012
:102F2000404041414141414040404040404040409C
:102F30004040404040404040400502020202020240
:102F4000020202020202020202202020202020208F
:102F500020202002020202020202909090909090A3
:102F60001010101010101010101010101010101061
:102F700010101010020202020202888888888888D5
:102F800008080808080808080808080808080808C1
:102F9000080808080202020240000000192F000081
:102FA0004E52465F4552524F525F494E56414C4930
:102FB000445F4441544100004E52465F4552524FD7
:102FC000525F534F46544445564943455F4E4F5414
:102FD0005F454E41424C4544000000004E52465F62
:102FE0004552524F525F464541545552455F4E4FF0
:102FF000545F454E41424C45440000004E52465FEE
:103000004552524F525F4D555445585F554E4C4FA7
:10301000434B5F4641494C45440000004E52465FD9
:103020004552524F525F4D555445585F4C4F434B9C
:103030005F4641494C4544004E52465F4552524F0F
:10304000525F4D555445585F434F4E445F494E497A
:10305000545F4641494C4544000000004E52465FD3
:103060004552524F525F4D555445585F494E495451
:103070005F4641494C4544004E52465F4552524FCF
:10308000525F424C455F495053505F52585F504B1E
:10309000545F5452554E4341544544004E52465F8E
:1030A0004552524F525F424C455F495053505F501A
:1030B0004545525F52454A4543544544000000008F
:1030C0004E52465F4552524F525F424C455F495007
:1030D00053505F4C494E4B5F444953434F4E4E450E
:1030E00043544544000000004E52465F4552524F43
:1030F000525F4150495F4E4F545F494D504C454DD2
:10310000454E5445440000004E52465F4552524FD2
:10311000525F4E4F545F535550504F5254454400E8
:103120004E52465F4552524F525F4D4F44554C45AB
:103130005F4E4F545F494E495449414C495A4544AA
:10314000000000004E52465F4552524F525F4D4FB5
:1031500044554C455F414C52454144595F494E49A5
:103160005449414C495A4544000000004E52465FC4
:103170004552524F525F4E4F545F464F554E44009A
:103180004E52465F4552524F525F494E56414C494E
:10319000445F5354415445004E52465F4552524F8E
:1031A000525F444154415F53495A45004E52465F75
:1031B0004552524F525F494F5F50454E44494E472A
:1031C000000000004E52465F4552524F525F535628
:1031D000435F48414E444C45525F4D495353494E1D
:1031E000470000004E52465F4552524F525F494ED3
:1031F00056414C49445F4C454E475448000000003E
:103200004E52465F4552524F525F4452565F54579A
:10321000495F4552525F414E41434B004E52465F1B
:103220004552524F525F4452565F5457495F455280
:10323000525F444E41434B004E52465F4552524FFF
:10324000525F494E5445524E414C00004E52465F2B
:103250004552524F525F53544F524147455F465576
:103260004C4C00004E52465F4552524F525F4E55F5
:103270004C4C00004E52465F4552524F525F494EF1
:1032800056414C49445F504152414D004E52465FB9
:103290004552524F525F4E4F5F4D454D000000006A
:1032A0004E52465F4552524F525F464F524249443A
:1032B00044454E004E52465F4552524F525F445273
:1032C000565F5457495F4552525F4F5645525255CB
:1032D0004E0000004E52465F4552524F525F494EDB
:1032E00056414C49445F4144445200004E52465FAF
:1032F0004552524F525F494E56414C49445F464CED
:10330000414753004E52465F535543434553530084
:103310004E52465F4552524F525F424C455F4950B4
:1033200053505F4348414E4E454C5F414C524541DE
:1033300044595F4558495354530000004E52465F6C
:103340004552524F525F54494D454F55540000006D
:103350004E52465F4552524F525F425553590000FC
:103360007761726E696E6700646562756700000060
:103370001B5B313B33306D001B5B306D0000000088
:103380001B5B313B33316D001B5B313B33326D00D6
:103390001B5B313B33336D001B5B313B33346D00C2
:1033A0001B5B313B33356D001B5B313B33366D00AE
:1033B0001B5B313B33376D00696E666F00000000A8
:1033C0006572726F720000005052530053414144C5
:1033D0004300000054494D455200000055415254ED
:1033E0000000000055415254450000007077725FA4
:1033F0006D676D740000000062616C6C6F632E6C11
:103400006F675F6D656D706F6F6C0000617070004D
:103410008834000000000020CC000000600800009C
:1034200054350000CC000020D425000070080000B6
:10343000C833000000000000CC3300000000000092
:10344000D433000000000000DC3300000000000066
:10345000E433000000000000EC3300000000000036
:10346000F8330000000000030C34000000000303E8
:10347000600000205800002060000020B8010020FB
:10348000C400002018000000000000000000000040
:10349000000000000000000000000000000000002C
:1034A000000000000000000000000000000000001C
:1034B000000000000000000000000000000000000C
:1034C000000000000020004000000000002000403C
:1034D00000000000EC2E00000000000000000000D2
:1034E00000000000000000000000000000000000DC
:1034F000000000000000000000000000C0330000D9
:1035000060330000B83300006833000078330000F7
:1035100070330000803300008833000090330000D7
:1035200098330000A0330000A8330000B03300003F
:103530000090D00300000000000000000000000028
:10354000000000000000000000000000000000007B
:043550000000000077
:0400000500000201F4
:00000001FF
